:03000000020030CB
:0300030002015E99
:03001B00020122BD
:10003000D29475891175A88975B808D28879007A23
:10004000007B007C007D007E00752000752100751E
:10005000220075230011BAD294517C09B90A1DBA45
:10006000051EBB0922BC0528BE023DBD032D79003B
:100070007A007B007C007D007E0011BA11BA80D727
:100080000A790011BA80D00B79007A0011BA80C7C2
:100090000C79007A007B0011BA80BC0D79007A00DF
:1000A0007B007C0011BA80AFBD09F00E79007A00A8
:1000B0007B007C007D0011BA809D7F327580FE89B7
:1000C000A011E97580FD8AA011E97580FB8BA01154
:1000D000E97580F78CA011E97580EF8DA011E975A5
:1000E00080DF8EA011E9DFD422758A48758CF4D2A6
:1000F0008C11FB308DFDC28CC28D22209011C293D9
:1001000030951EC295758D00758B00D28E801220A1
:10011000910F30950CC295758B00758D00D28E8035
:1001200000223094028003020208209317BB0905C5
:100130000C7B0080010BBC06047B007C00D293C2C8
:100140008ED29532BE0209BD030E7E007D0080096D
:10015000BD09050E7D0080010DC28ED29532C2947C
:1001600009B90A1FBA0520BB0924BC052ABE023FF3
:10017000BD032F79007A007B007C007D007E00317A
:10018000C180DD31C180D90A790031C180D20B79BB
:10019000007A0031C180C90C79007A007B0031C13E
:1001A00080BE0D79007A007B007C0031C180B1BD3A
:1001B00009F00E79007A007B007C007D0031C1805F
:1001C0009F7F327580FE75A00031F67580FD75A0A9
:1001D0000031F67580FB8520A031F67580F785210A
:1001E000A031F67580EF8522A031F67580DF85237A
:1001F000A031F6DFCE22758A48758CF4D28C511767
:10020000308DFDC28CC28D2220934CE520B4093381
:100210000521752000802E209011C293309523C2B5
:1002200095758B00758D00D28E801720910F3095BB
:1002300011C295758B00758D00D28E8005209202BB
:100240008050220520E521B40606752000752100A6
:10025000D293C28ED29532E523B4020DE522B403C7
:1002600014752300752200800EE522B409070523CA
:1002700075220080020522C28ED29532EBB5200F86
:10028000ECB5210BEDB52207EEB52303C29622D2C1
:0C0290009622758150755157755200324E
:00000001FF
